 SwiGobi

 Timestamp is 54003a01 (Fri Aug 29 16:29:53 2014)

 Preferred load address is 10000000

 Start         Length     Name                   Class
 0001:00000000 000372e8H .text                   CODE
 0001:000372e8 0000006cH .text$yc                CODE
 0001:00037354 00000014H .text$yd                CODE
 0002:00000000 00021b98H .rdata                  DATA
 0002:00021b98 00000070H .rdata$debug            DATA
 0002:00021c08 00000168H .xdata                  DATA
 0002:00021d70 0000003cH .idata$2                DATA
 0002:00021dac 00000014H .idata$3                DATA
 0002:00021dc0 00000224H .idata$4                DATA
 0002:00021fe4 000002d6H .idata$6                DATA
 0002:000222c0 0000035fH .edata                  DATA
 0003:00000000 00000224H .idata$5                DATA
 0003:00000224 00000004H .CRT$XCA                DATA
 0003:00000228 00000004H .CRT$XCAA               DATA
 0003:0000022c 00000004H .CRT$XCU                DATA
 0003:00000230 00000004H .CRT$XCZ                DATA
 0003:00000234 00000004H .CRT$XIA                DATA
 0003:00000238 00000004H .CRT$XIZ                DATA
 0003:0000023c 00000004H .CRT$XPA                DATA
 0003:00000240 00000004H .CRT$XPZ                DATA
 0003:00000244 00000004H .CRT$XTA                DATA
 0003:00000248 00000004H .CRT$XTZ                DATA
 0003:00000250 00000784H .data                   DATA
 0003:000009d8 00002c98H .bss                    DATA
 0004:00000000 00000dd8H .pdata                  DATA
 0005:00000000 00000058H .rsrc$01                DATA
 0005:00000060 000003f0H .rsrc$02                DATA

  Address         Publics by Value              Rva+Base       Lib:Object

 0000:00000000       ___safe_se_handler_table   00000000     <absolute>
 0000:00000000       ___safe_se_handler_count   00000000     <absolute>
 0001:00000000       ?ThreadFunc@@YAKPAX@Z      10001000 f   CEPowerControl.obj
 0001:00000040       ??0CCEPowerControl@@QAA@P6AHHHPAX@ZH00@Z 10001040 f   CEPowerControl.obj
 0001:000002cc       ??1CCEPowerControl@@QAA@XZ 100012cc f   CEPowerControl.obj
 0001:000003f4       ?NotifyDeviceRemoved@CCEPowerControl@@QAAXXZ 100013f4 f   CEPowerControl.obj
 0001:00000470       ?MonitorSystemPowerState@CCEPowerControl@@QAAXXZ 10001470 f   CEPowerControl.obj
 0001:00000f98       ?WaitForSingleObjectReset@CCEPowerControl@@QAAKPAXK@Z 10001f98 f   CEPowerControl.obj
 0001:000010bc       ?ProcessPowerNotification@CCEPowerControl@@AAAXPAX@Z 100020bc f   CEPowerControl.obj
 0001:00001260       SetEvent                   10002260 f i CEPowerControl.obj
 0001:00001294       ResetEvent                 10002294 f i CEPowerControl.obj
 0001:000012c8       ??0CircularBuffer@@QAA@XZ  100022c8 f   circularbuffer.obj
 0001:00001338       ??1CircularBuffer@@QAA@XZ  10002338 f   circularbuffer.obj
 0001:00001350       ?Write@CircularBuffer@@QAAHPAEI@Z 10002350 f   circularbuffer.obj
 0001:000017b8       ?Write@CircularBuffer@@QAAHPAEI0I@Z 100027b8 f   circularbuffer.obj
 0001:00001d34       ?HasData@CircularBuffer@@QAAHXZ 10002d34 f   circularbuffer.obj
 0001:00001db8       ?DataBytesInBuffer@CircularBuffer@@QAAKXZ 10002db8 f   circularbuffer.obj
 0001:00001e34       ?SpaceInBuffer@CircularBuffer@@QAAKXZ 10002e34 f   circularbuffer.obj
 0001:00001ec0       ?ResetBuffer@CircularBuffer@@QAAXXZ 10002ec0 f   circularbuffer.obj
 0001:00001f20       ?Read@CircularBuffer@@QAAHPAEIPAI@Z 10002f20 f   circularbuffer.obj
 0001:000023e4       ?Init@CircularBuffer@@QAAXIH@Z 100033e4 f   circularbuffer.obj
 0001:00002570       ?GetBufferReadPosition@CircularBuffer@@QAAKXZ 10003570 f   circularbuffer.obj
 0001:00002638       ?GetBufferWritePosition@CircularBuffer@@QAAKXZ 10003638 f   circularbuffer.obj
 0001:00002700       ?GetBufferSize@CircularBuffer@@QAAKXZ 10003700 f   circularbuffer.obj
 0001:0000276c       ?DeInit@CircularBuffer@@QAAXXZ 1000376c f   circularbuffer.obj
 0001:00002814       ?DevicePowerNotify@@YAHHHPAX@Z 10003814 f   commdevice.obj
 0001:00002948       ??0CommDevice@@QAA@PB_W@Z  10003948 f   commdevice.obj
 0001:00002be4       ??1CommDevice@@UAA@XZ      10003be4 f   commdevice.obj
 0001:00002ce8       ?ReOpen@CommDevice@@QAAKXZ 10003ce8 f   commdevice.obj
 0001:00002e84       ?Open@CommDevice@@QAAKKKH@Z 10003e84 f   commdevice.obj
 0001:0000352c       ?Close@CommDevice@@QAAHH@Z 1000452c f   commdevice.obj
 0001:000039e4       ?Read@CommDevice@@QAAKPAXK@Z 100049e4 f   commdevice.obj
 0001:00003dc0       ?Write@CommDevice@@QAAKPBXK@Z 10004dc0 f   commdevice.obj
 0001:000041c4       ?PowerUp@CommDevice@@QAAXXZ 100051c4 f   commdevice.obj
 0001:000041d4       ?PowerDown@CommDevice@@QAAXXZ 100051d4 f   commdevice.obj
 0001:000041e4       ?Seek@CommDevice@@QAAKJG@Z 100051e4 f   commdevice.obj
 0001:00004208       ?IoControl@CommDevice@@QAAHKPAEK0KPAK@Z 10005208 f   commdevice.obj
 0001:00004dc4       ?CardRemovedNotify@CommDevice@@AAAXH@Z 10005dc4 f   commdevice.obj
 0001:00004e64       ?SetHostJustResumedEvent@CommDevice@@QAAXXZ 10005e64 f   commdevice.obj
 0001:00004ebc       ?GetPortNumber@CommDevice@@QAAKXZ 10005ebc f   commdevice.obj
 0001:00004ee8       ?DeInitPowerControl@CommDevice@@QAAXXZ 10005ee8 f   commdevice.obj
 0001:00004ff8       ?LogCritical@@YAXPA_WZZ    10005ff8 f i commdevice.obj
 0001:000050a0       ??_ECommDevice@@UAAPAXI@Z  100060a0 f i commdevice.obj
 0001:000050a0       ??_GCommDevice@@UAAPAXI@Z  100060a0 f i commdevice.obj
 0001:000050e0       PulseEvent                 100060e0 f i commdevice.obj
 0001:00005114       ??_GCCEPowerControl@@QAAPAXI@Z 10006114 f i commdevice.obj
 0001:00005154       ??_GCPPP4pcap@@QAAPAXI@Z   10006154 f i commdevice.obj
 0001:0000519c       ?WMP_Init@@YAKPB_WPBX@Z    1000619c f   commentry.obj
 0001:00005250       ?WMP_Deinit@@YAHK@Z        10006250 f   commentry.obj
 0001:000052f8       ?WMP_Open@@YAKKKK@Z        100062f8 f   commentry.obj
 0001:0000537c       ?WMP_Close@@YAHK@Z         1000637c f   commentry.obj
 0001:000053e0       ?WMP_Read@@YAKKPAXK@Z      100063e0 f   commentry.obj
 0001:00005420       ?WMP_Write@@YAKKPBXK@Z     10006420 f   commentry.obj
 0001:00005460       ?WMP_Seek@@YAKKJG@Z        10006460 f   commentry.obj
 0001:0000548c       ?WMP_PowerDown@@YAXK@Z     1000648c f   commentry.obj
 0001:000054c4       ?WMP_PowerUp@@YAXK@Z       100064c4 f   commentry.obj
 0001:0000550c       ?WMP_IOControl@@YAHKKPAEK0KPAK@Z 1000650c f   commentry.obj
 0001:00005568       ??0CtlService@@QAA@XZ      10006568 f   CtlService.obj
 0001:00005670       ??1CtlService@@UAA@XZ      10006670 f   CtlService.obj
 0001:000056d0       ?Initialize@CtlService@@QAA_NPAUQMI_CHANNEL@@@Z 100066d0 f   CtlService.obj
 0001:000057d0       ?Shutdown@CtlService@@QAAXXZ 100067d0 f   CtlService.obj
 0001:000058b4       ?ProcessSynchronousTransaction@CtlService@@QAAHPAVCtlTransaction@@GK@Z 100068b4 f   CtlService.obj
 0001:00005c64       ?HandleTransactionResponse@CtlService@@IAAXPAEG@Z 10006c64 f   CtlService.obj
 0001:00005d74       ?HandleTransactionIndication@CtlService@@IAAXPAEG@Z 10006d74 f   CtlService.obj
 0001:00005d84       ?ReadNotify@CtlService@@QAAXPAEG@Z 10006d84 f   CtlService.obj
 0001:00005e00       ?NewTransactionId@CtlService@@IAAEXZ 10006e00 f   CtlService.obj
 0001:00005ea0       ?AddToOutstandingList@CtlService@@IAAXPAVCtlTransaction@@@Z 10006ea0 f   CtlService.obj
 0001:00005f24       ?RemoveFromOutstandingList@CtlService@@IAAXPAVCtlTransaction@@@Z 10006f24 f   CtlService.obj
 0001:00005f90       ?AddToFreeList@CtlService@@QAAXPAVCtlTransaction@@@Z 10006f90 f   CtlService.obj
 0001:00006014       ?RemoveFromFreeList@CtlService@@IAAXPAVCtlTransaction@@@Z 10007014 f   CtlService.obj
 0001:00006080       ?GetFromFreeList@CtlService@@QAAPAVCtlTransaction@@XZ 10007080 f   CtlService.obj
 0001:000060ec       ??0CtlTransaction@@QAA@XZ  100070ec f i CtlService.obj
 0001:00006154       ??1CtlTransaction@@QAA@XZ  10007154 f i CtlService.obj
 0001:00006174       ??_GCtlService@@UAAPAXI@Z  10007174 f i CtlService.obj
 0001:00006174       ??_ECtlService@@UAAPAXI@Z  10007174 f i CtlService.obj
 0001:000061b4       RemoveTailList             100071b4 f i CtlService.obj
 0001:00006224       ??0DmsService@@QAA@XZ      10007224 f   DmsService.obj
 0001:00006330       ??1DmsService@@UAA@XZ      10007330 f   DmsService.obj
 0001:00006394       ?Initialize@DmsService@@QAA_NPAUQMI_CHANNEL@@E@Z 10007394 f   DmsService.obj
 0001:000064b4       ?Shutdown@DmsService@@QAAXXZ 100074b4 f   DmsService.obj
 0001:00006598       ?ProcessSynchronousTransaction@DmsService@@QAAHPAVQmiTransaction@@GK@Z 10007598 f   DmsService.obj
 0001:00006828       ?HandleTransactionResponse@DmsService@@IAAXPAEG@Z 10007828 f   DmsService.obj
 0001:00006960       ?HandleTransactionIndication@DmsService@@IAAXPAEG@Z 10007960 f   DmsService.obj
 0001:00006970       ?ReadNotify@DmsService@@QAAXPAEG@Z 10007970 f   DmsService.obj
 0001:000069ec       ?NewTransactionId@DmsService@@IAAGXZ 100079ec f   DmsService.obj
 0001:00006a94       ?AddToOutstandingList@DmsService@@IAAXPAVQmiTransaction@@@Z 10007a94 f   DmsService.obj
 0001:00006b18       ?RemoveFromOutstandingList@DmsService@@IAAXPAVQmiTransaction@@@Z 10007b18 f   DmsService.obj
 0001:00006b84       ?AddToFreeList@DmsService@@QAAXPAVQmiTransaction@@@Z 10007b84 f   DmsService.obj
 0001:00006c08       ?RemoveFromFreeList@DmsService@@IAAXPAVQmiTransaction@@@Z 10007c08 f   DmsService.obj
 0001:00006c74       ?GetFromFreeList@DmsService@@QAAPAVQmiTransaction@@XZ 10007c74 f   DmsService.obj
 0001:00006ce0       ??0QmiTransaction@@QAA@XZ  10007ce0 f i DmsService.obj
 0001:00006d68       ??1QmiTransaction@@QAA@XZ  10007d68 f i DmsService.obj
 0001:00006d88       ??_GDmsService@@UAAPAXI@Z  10007d88 f i DmsService.obj
 0001:00006d88       ??_EDmsService@@UAAPAXI@Z  10007d88 f i DmsService.obj
 0001:00006dc8       ?WceOpen@@YAXXZ            10007dc8 f   dpwce.obj
 0001:00006e50       ?WceClose@@YAXXZ           10007e50 f   dpwce.obj
 0001:00006e84       ?WcePutString@@YAXPADH@Z   10007e84 f   dpwce.obj
 0001:00006ed0       ?DpPrint@@YAXPADZZ         10007ed0 f   dpwce.obj
 0001:00006fe4       ?dp_print_buffer@@YAXPBD0H@Z 10007fe4 f   dpwce.obj
 0001:00007284       ?dp_print_buffer16@@YAXPBD00H@Z 10008284 f   dpwce.obj
 0001:000073e4       ?PMInitialize@@YAHXZ       100083e4 f   pmcommon.obj
 0001:00007428       ?PMShutdown@@YAXPAUsAdapterConfig@@@Z 10008428 f   pmcommon.obj
 0001:00007458       ?time4PPPLog@@YAEPAK@Z     10008458 f   PPP4pcap.obj
 0001:00007530       ??0CPPP4pcap@@QAA@K@Z      10008530 f   PPP4pcap.obj
 0001:0000760c       ??1CPPP4pcap@@QAA@XZ       1000860c f   PPP4pcap.obj
 0001:00007668       ?WriteLogFile@CPPP4pcap@@QAAKKPBXK@Z 10008668 f   PPP4pcap.obj
 0001:000078e8       ?WriteNewTime@CPPP4pcap@@QAAKK@Z 100088e8 f   PPP4pcap.obj
 0001:00007a00       ?qlIsListEmpty@@YAEPAU_LIST_ENTRY@@@Z 10008a00 f   qlmanage.obj
 0001:00007a50       ?qlremovenext@@YAPAU_LIST_ENTRY@@PAU1@PAU_NDIS_SPIN_LOCK@@@Z 10008a50 f   qlmanage.obj
 0001:00007b34       ?qlinserttail@@YAXPAU_LIST_ENTRY@@PAU_NDIS_SPIN_LOCK@@0@Z 10008b34 f   qlmanage.obj
 0001:00007bf0       ?qlinserthead@@YAXPAU_LIST_ENTRY@@PAU_NDIS_SPIN_LOCK@@0@Z 10008bf0 f   qlmanage.obj
 0001:00007ca8       ?qlremovenext_signalnotempty@@YAPAU_LIST_ENTRY@@PAU1@PAU_NDIS_SPIN_LOCK@@PAU_NDIS_EVENT@@@Z 10008ca8 f   qlmanage.obj
 0001:00007dc8       ?qlinserttail_signalnotempty@@YAXPAU_LIST_ENTRY@@PAU_NDIS_SPIN_LOCK@@0PAU_NDIS_EVENT@@@Z 10008dc8 f   qlmanage.obj
 0001:00007e94       ?RetrieveVersionInfo@@YAHPAU_QMICTL_GET_VERSION_RESP_MSG@@@Z 10008e94 f   qmi.obj
 0001:00008508       ?GetQMIVersions@@YAHXZ     10009508 f   qmi.obj
 0001:000086c0       ?GetClientID@@YAHW4_QMI_SERVICE_TYPE@@PAEPAW4_QMI_ERROR_CODE_TYPE@@@Z 100096c0 f   qmi.obj
 0001:000088e4       ?ReleaseClientID@@YAHW4_QMI_SERVICE_TYPE@@E@Z 100098e4 f   qmi.obj
 0001:00008b18       ?DmsGetDeviceManufacturer@@YAHPADH@Z 10009b18 f   qmi.obj
 0001:00008d30       ?DmsGetDeviceMsisdn@@YAHPADH@Z 10009d30 f   qmi.obj
 0001:00008f48       ?WdsSetEventReportIndicationCallback@@YAXP6AXPAXPAEG@Z0@Z 10009f48 f   qmi.obj
 0001:00008f70       ?WdsSetEventReportAsync@@YAHHP6AXPAXPAEG@Z0@Z 10009f70 f   qmi.obj
 0001:00009160       ?WdsSetGetPacketServiceStatusIndicationCallbackCallback@@YAXP6AXPAXPAEG@Z0@Z 1000a160 f   qmi.obj
 0001:00009188       ?WdsGetCurrentChannelRate@@YAHPAK000@Z 1000a188 f   qmi.obj
 0001:00009418       ?SendQMIMessage@@YAKPAUQMI_CHANNEL@@PAEGEW4_QMI_SERVICE_TYPE@@@Z 1000a418 f   qmi.obj
 0001:00009540       ?ConfigPowerSaveSetting@@YAHKGEPAGPAW4_QMI_ERROR_CODE_TYPE@@@Z 1000a540 f   qmi.obj
 0001:0000987c       ?SetPowerSaveMode@@YAHK@Z  1000a87c f   qmi.obj
 0001:00009a90       ?GetPowerSaveMode@@YAHPAKPAW4_QMI_ERROR_CODE_TYPE@@@Z 1000aa90 f   qmi.obj
 0001:00009d24       ?QMI_Init@@YAPAXPB_WPBX@Z  1000ad24 f   qmicom.obj
 0001:0000a000       ?QMI_Open@@YAPAXPAXKK@Z    1000b000 f   qmicom.obj
 0001:0000aaa4       ?QMI_Close@@YAHPAUQMI_OPEN_INFO@@@Z 1000baa4 f   qmicom.obj
 0001:0000aef0       ?QMI_Deinit@@YAHPAUQMI_PORT_MDD@@@Z 1000bef0 f   qmicom.obj
 0001:0000b03c       ?QMI_Read@@YAKPAXPAEK@Z    1000c03c f   qmicom.obj
 0001:0000b3bc       ?QMI_Write@@YAKPAXPAEK@Z   1000c3bc f   qmicom.obj
 0001:0000b768       ?QMI_Seek@@YAKPAXJK@Z      1000c768 f   qmicom.obj
 0001:0000b78c       ?QMI_PowerUp@@YAHPAX@Z     1000c78c f   qmicom.obj
 0001:0000b7ec       ?QMI_PowerDown@@YAHPAX@Z   1000c7ec f   qmicom.obj
 0001:0000b84c       ?QMI_IOControl@@YAHPAUQMI_OPEN_INFO@@KPAEK1KPAK@Z 1000c84c f   qmicom.obj
 0001:0000c54c       ?EvaluateEventFlag@@YAXPAUQMI_PORT_MDD@@K@Z 1000d54c f   qmicom.obj
 0001:0000c854       ?QmiUpdateSerialState@@YAXPAUQMI_PORT_MDD@@K@Z 1000d854 f   qmicom.obj
 0001:0000c894       ?QmiSetSerialStatusState@@YAXPAUQMI_PORT_MDD@@EEEEG@Z 1000d894 f   qmicom.obj
 0001:0000cb34       ?QmiAddToReadQueue@@YAEPAUQMI_PORT_MDD@@PAEK@Z 1000db34 f   qmicom.obj
 0001:0000cdcc       ?QmiWaitCommEvent@@YAHPAUQMI_OPEN_INFO@@PAKPAU_OVERLAPPED@@@Z 1000ddcc f   qmicom.obj
 0001:0000e7f0       ?ProcessClientMsg@@YAXPAUQMI_OPEN_INFO@@PAEK@Z 1000f7f0 f   qmicom.obj
 0001:0000e870       ??0RilOutContextPool@@QAA@XZ 1000f870 f   RilOutContextPool.obj
 0001:0000eaf8       ??1RilOutContextPool@@UAA@XZ 1000faf8 f   RilOutContextPool.obj
 0001:0000eb4c       ?SetContextId@RilOutContextPool@@QAAXK@Z 1000fb4c f   RilOutContextPool.obj
 0001:0000eb70       ?SetStatusCallback@RilOutContextPool@@QAAXP6AXPAXPAUrilndisstatus_tag@@@Z0@Z 1000fb70 f   RilOutContextPool.obj
 0001:0000eba8       ?Allocate@RilOutContextPool@@QAAPAURilOutContext@@XZ 1000fba8 f   RilOutContextPool.obj
 0001:0000ee60       ?Free@RilOutContextPool@@QAAXPAURilOutContext@@@Z 1000fe60 f   RilOutContextPool.obj
 0001:0000f078       ?DumpList@RilOutContextPool@@QAAXXZ 10010078 f   RilOutContextPool.obj
 0001:0000f138       ?AddToPendingList@RilOutContextPool@@QAAXPAURilOutContext@@@Z 10010138 f   RilOutContextPool.obj
 0001:0000f1f4       ?RemoveFromToPendingList@RilOutContextPool@@QAAPAURilOutContext@@XZ 100101f4 f   RilOutContextPool.obj
 0001:0000f35c       ??_ERilOutContextPool@@UAAPAXI@Z 1001035c f i RilOutContextPool.obj
 0001:0000f35c       ??_GRilOutContextPool@@UAAPAXI@Z 1001035c f i RilOutContextPool.obj
 0001:0000f39c       ??0RilPacketPool@@QAA@XZ   1001039c f   RilPacketPool.obj
 0001:0000f63c       ??1RilPacketPool@@UAA@XZ   1001063c f   RilPacketPool.obj
 0001:0000f670       ?SetContextId@RilPacketPool@@QAAXK@Z 10010670 f   RilPacketPool.obj
 0001:0000f6c0       ?Allocate@RilPacketPool@@QAAPAUrilndispacket_tag@@XZ 100106c0 f   RilPacketPool.obj
 0001:0000f8b8       ?Free@RilPacketPool@@QAAXPAUrilndispacket_tag@@@Z 100108b8 f   RilPacketPool.obj
 0001:0000f9d4       ?DumpList@RilPacketPool@@QAAXXZ 100109d4 f   RilPacketPool.obj
 0001:0000faa4       ??_ERilPacketPool@@UAAPAXI@Z 10010aa4 f i RilPacketPool.obj
 0001:0000faa4       ??_GRilPacketPool@@UAAPAXI@Z 10010aa4 f i RilPacketPool.obj
 0001:0000faec       ?SWD_Init@@YAPAXPB_WPBX@Z  10010aec f   swdcom.obj
 0001:0000fe10       ?SWD_Open@@YAPAXPAXKK@Z    10010e10 f   swdcom.obj
 0001:000100e0       ?SWD_Close@@YAHPAUSWD_OPEN_INFO@@@Z 100110e0 f   swdcom.obj
 0001:000102f4       ?SWD_Deinit@@YAHPAUSWD_MDD@@@Z 100112f4 f   swdcom.obj
 0001:00010490       ?SWD_Read@@YAKPAXPAEK@Z    10011490 f   swdcom.obj
 0001:000104b4       ?SWD_Write@@YAKPAXPAEK@Z   100114b4 f   swdcom.obj
 0001:000104d8       ?SWD_Seek@@YAKPAXJK@Z      100114d8 f   swdcom.obj
 0001:000104fc       ?SWD_PowerUp@@YAHPAX@Z     100114fc f   swdcom.obj
 0001:00010520       ?SWD_PowerDown@@YAHPAX@Z   10011520 f   swdcom.obj
 0001:00010544       ?SWD_IOControl@@YAHPAUSWD_OPEN_INFO@@KPAEK1KPAK@Z 10011544 f   swdcom.obj
 0001:00010a84       ?ReadDWORDValue@@YAJPAUHKEY__@@PB_W1PAK@Z 10011a84 f   swicom.obj
 0001:00010b68       ?WriteDWORDValue@@YAJPAUHKEY__@@PB_W1K@Z 10011b68 f   swicom.obj
 0001:00010c74       ?ReadStrValue@@YAJPAUHKEY__@@PB_W1QA_WK@Z 10011c74 f   swicom.obj
 0001:00010d74       ?WriteStrValue@@YAJPAUHKEY__@@PB_W1QA_WK@Z 10011d74 f   swicom.obj
 0001:00010e80       DllMain                    10011e80 f   swicom.obj
 0001:00011040       ?dumpBytesData@@YAXKPA_WPAEK@Z 10012040 f   swicom.obj
 0001:00011450       ?initDefaultDCB@@YAXPAU_DCB@@@Z 10012450 f   swicom.obj
 0001:000116d0       ?initDefaultCommProp@@YAXPAU_COMMPROP@@@Z 100126d0 f   swicom.obj
 0001:000117d8       ?IsSystemCleanBooting@@YAHXZ 100127d8 f   swicom.obj
 0001:00011854       ?SWI_Init@@YAPAXPB_WPBX@Z  10012854 f   swicom.obj
 0001:00011b58       ?PortStatusIsOpen@@YAEPAUVSP_OPEN_INFO@@H@Z 10012b58 f   swicom.obj
 0001:00011c1c       ?PortStatusOpen@@YAXPAUVSP_OPEN_INFO@@@Z 10012c1c f   swicom.obj
 0001:00011ca0       ?PortStatusClose@@YAXPAUVSP_OPEN_INFO@@@Z 10012ca0 f   swicom.obj
 0001:00011d30       ?SWI_Open@@YAPAXPAXKK@Z    10012d30 f   swicom.obj
 0001:00012b34       ?SWI_Close@@YAHPAUVSP_OPEN_INFO@@@Z 10013b34 f   swicom.obj
 0001:000131f0       ?SWI_Deinit@@YAHPAUVSP_PORT_MDD@@@Z 100141f0 f   swicom.obj
 0001:00013388       ?SWI_Read@@YAKPAXPAEK@Z    10014388 f   swicom.obj
 0001:00013600       ?SWI_Write@@YAKPAXPAEK@Z   10014600 f   swicom.obj
 0001:00013b28       ?SWI_Seek@@YAKPAXJK@Z      10014b28 f   swicom.obj
 0001:00013b4c       ?SWI_PowerUp@@YAHPAX@Z     10014b4c f   swicom.obj
 0001:00013bac       ?SWI_PowerDown@@YAHPAX@Z   10014bac f   swicom.obj
 0001:00013c14       ?DbgPrintEventMask@@YAXK@Z 10014c14 f   swicom.obj
 0001:00013fa8       ?SWI_IOControl@@YAHPAUVSP_OPEN_INFO@@KPAEK1KPAK@Z 10014fa8 f   swicom.obj
 0001:000150d4       ?EvaluateEventFlag@@YAXPAUVSP_PORT_MDD@@K@Z 100160d4 f   swicom.obj
 0001:000153d8       ?VspUpdateSerialState@@YAXPAUVSP_PORT_MDD@@K@Z 100163d8 f   swicom.obj
 0001:00015418       ?VspSetSerialStatusState@@YAXPAUVSP_PORT_MDD@@EEEEG@Z 10016418 f   swicom.obj
 0001:000156b8       ?VspAddToReadQueue@@YAEPAUVSP_PORT_MDD@@PAEK@Z 100166b8 f   swicom.obj
 0001:00015950       ?VspWaitCommEvent@@YAHPAUVSP_OPEN_INFO@@PAKPAU_OVERLAPPED@@@Z 10016950 f   swicom.obj
 0001:0001756c       ?GetAvailStoreMem@@YAKXZ   1001856c f   swiroutines.obj
 0001:00017600       ?GetMemUsed@@YAKXZ         10018600 f   swiroutines.obj
 0001:00017634       ?UnblockAllChannelThread@@YAXXZ 10018634 f   swiroutines.obj
 0001:0001765c       ?OpenOutModemBulkPipe11@@YAPAXU_USB_ENDPOINT_DESCRIPTOR@@@Z 1001865c f   swiroutines.obj
 0001:0001771c       ?CloseModemPipe@@YAHPAX@Z  1001871c f   swiroutines.obj
 0001:000177c0       ?OpenInModemBulkPipe10@@YAPAXU_USB_ENDPOINT_DESCRIPTOR@@@Z 100187c0 f   swiroutines.obj
 0001:00017880       ?DataXferModemBulkPipe11@@YAPAXPAXPAEK@Z 10018880 f   swiroutines.obj
 0001:00017910       ?EnableModemRemoteWakeup@@YAXXZ 10018910 f   swiroutines.obj
 0001:00017c5c       ?DisableModemRemoteWakeup@@YAXXZ 10018c5c f   swiroutines.obj
 0001:00017f60       ?ModemPowerD0@@YAXXZ       10018f60 f   swiroutines.obj
 0001:000181d8       ?ModemPowerD1@@YAXXZ       100191d8 f   swiroutines.obj
 0001:00018450       ?ModemPowerD2@@YAXXZ       10019450 f   swiroutines.obj
 0001:000186c8       ?ModemPowerD3@@YAXXZ       100196c8 f   swiroutines.obj
 0001:00018944       ?DoSendInitControlRequests@@YAHKKH@Z 10019944 f   swiroutines.obj
 0001:00018fc8       ?SendInitControlRequests@@YAHKKH@Z 10019fc8 f   swiroutines.obj
 0001:000190e0       ?OpenInterruptModemPipe1@@YAPAXU_USB_ENDPOINT_DESCRIPTOR@@@Z 1001a0e0 f   swiroutines.obj
 0001:0001918c       ?SWIUSBPowerControl@@YAHHHPAH@Z 1001a18c f   swiroutines.obj
 0001:000194fc       ?UsbGetMuxMode@@YAHPAW4_MUX_INSTANCE_STATE@@@Z 1001a4fc f   swiroutines.obj
 0001:00019618       ?UsbSetMuxMode@@YAHPAU_MUX_MODE_PARAMETERS@@@Z 1001a618 f   swiroutines.obj
 0001:00019768       ?UsbSetNmxMode@@YAHXZ      1001a768 f   swiroutines.obj
 0001:000197dc       ?UsbGetNMEAMode@@YAHPAG@Z  1001a7dc f   swiroutines.obj
 0001:00019858       ?UsbSetNMEAMode@@YAHG@Z    1001a858 f   swiroutines.obj
 0001:000198d4       ?UsbSetHostSleepPowerState@@YAHG@Z 1001a8d4 f   swiroutines.obj
 0001:00019ba0       ?UsbGetAttributes@@YAHPAG@Z 1001aba0 f   swiroutines.obj
 0001:00019c34       ?SendHostToInterfaceCommandSync@@YAHPAU_USB_DEVICE_REQUEST@@PAEKK@Z 1001ac34 f   swiroutines.obj
 0001:00019ef8       ?SWICreateMemory@@YAPAEK@Z 1001aef8 f   swiroutines.obj
 0001:0001a0fc       ?SWIFreeMemory@@YAXPAE@Z   1001b0fc f   swiroutines.obj
 0001:0001a374       ?IsQMIChannelBusy@@YAHXZ   1001b374 f   swiroutines.obj
 0001:0001a470       ?HwIsModemBusy@@YAEPAU_SW_MODEM@@@Z 1001b470 f   swiroutines.obj
 0001:0001a644       ?EnsurePortResumed@@YAHK@Z 1001b644 f   swiroutines.obj
 0001:0001a800       ?GetDescriptor@@YAHEEGPAEGPAK@Z 1001b800 f   swiroutines.obj
 0001:0001a990       ?HandleInvalidModem@@YAXGG@Z 1001b990 f   swiroutines.obj
 0001:0001a9e0       ?SendSyncGPSCommand@@YAHPAUVSP_PORT_MDD@@W4_GPS_CMD@@@Z 1001b9e0 f   swiroutines.obj
 0001:0001abcc       GetCurrentThreadId         1001bbcc f i swiroutines.obj
 0001:0001abec       ?WaitForAllUsbThreadsReady@@YAEI@Z 1001bbec f   swiusb.obj
 0001:0001ae00       ?TransferCompletionRoutine@@YAKPAX@Z 1001be00 f   swiusb.obj
 0001:0001aed0       ?DispatchQMIMsg@@YAXPAEG@Z 1001bed0 f   swiusb.obj
 0001:0001b398       ?QMIThread@@YAXPAPAX@Z     1001c398 f   swiusb.obj
 0001:0001bc94       ?StartQMIThreads@@YAXXZ    1001cc94 f   swiusb.obj
 0001:0001bcf8       ?InitializeQMIChannel@@YAHE@Z 1001ccf8 f   swiusb.obj
 0001:0001bfc4       ?CleanupQMIChannel@@YAXXZ  1001cfc4 f   swiusb.obj
 0001:0001c2ac       ?InitializeDirectIpChannel@@YAHPBU_USB_INTERFACE@@PA_W@Z 1001d2ac f   swiusb.obj
 0001:0001d03c       ?CleanupDirectIpChannel@@YAXXZ 1001e03c f   swiusb.obj
 0001:0001d42c       ?StartDmsService@@YAHXZ    1001e42c f   swiusb.obj
 0001:0001d668       ?StopDmsService@@YAXXZ     1001e668 f   swiusb.obj
 0001:0001d71c       ?StartWdsService@@YAHXZ    1001e71c f   swiusb.obj
 0001:0001d958       ?StopWdsService@@YAXXZ     1001e958 f   swiusb.obj
 0001:0001da04       ?SWIResetPipe@@YAHPBU_USB_FUNCS@@PAX@Z 1001ea04 f   swiusb.obj
 0001:0001daa8       ?CreateRegistryPath@@YAXPA_WKPBU_USB_DRIVER_SETTINGS@@@Z 1001eaa8 f   swiusb.obj
 0001:0001dc54       ?SetDeviceStateActive@@YAXH@Z 1001ec54 f   swiusb.obj
 0001:0001dde0       ?SetUSBActivityEvent@@YAXXZ 1001ede0 f   swiusb.obj
 0001:0001de20       ?SetDeviceStateInActive@@YAXH@Z 1001ee20 f   swiusb.obj
 0001:000213fc       ?RilNdisReceivePacketDone@@YAXQAUrilndispacket_tag@@@Z 100223fc f   swiusb.obj
 0001:000214b0       ?TransmitRilPacketComplete@@YAKPAX@Z 100224b0 f   swiusb.obj
 0001:00021724       ?RilNdisSendPacket@@YAXQAUrilndispacket_tag@@@Z 10022724 f   swiusb.obj
 0001:000228b0       ?processMsmSerialState@@YAXPAU_SW_MODEM@@PADK@Z 100238b0 f   swiusb.obj
 0001:00023c10       ?DisplayMemoryStatus@@YAXXZ 10024c10 f   swiusb.obj
 0001:00023c70       ?USBDeviceNotifications@@YAHPAXKPAPAK111@Z 10024c70 f   swiusb.obj
 0001:0002492c       ?WMWdsGetPacketServiceStatusInd@@YAXPAXPAEG@Z 1002592c f   swiusb.obj
 0001:00024978       USBDeviceAttach            10025978 f   swiusb.obj
 0001:0002c014       USBInstallDriver           1002d014 f   swiusb.obj
 0001:0002c064       ?GetDeviceInstalledEvent@@YAPAXXZ 1002d064 f   swiusb.obj
 0001:0002c084       ?HookUsbToAdapter@@YAXPAUsAdapterConfig@@@Z 1002d084 f   swiusb.obj
 0001:0002c11c       ?HelpResumingOS@@YAKPAPAX@Z 1002d11c f   swiusb.obj
 0001:0002c194       ?ActivityThread@@YAXPAPAX@Z 1002d194 f   swiusb.obj
 0001:0002d950       ??0QMI_CHANNEL@@QAA@XZ     1002e950 f i swiusb.obj
 0001:0002d984       ??1_SW_MODEM@@QAA@XZ       1002e984 f i swiusb.obj
 0001:0002d9a0       ??1QMI_CHANNEL@@QAA@XZ     1002e9a0 f i swiusb.obj
 0001:0002d9bc       ??0WdsService@@QAA@XZ      1002e9bc f   WdsService.obj
 0001:0002db08       ??1WdsService@@UAA@XZ      1002eb08 f   WdsService.obj
 0001:0002db6c       ?SetEventReportIndicationCallback@WdsService@@QAAXP6AXPAXPAEG@Z0@Z 1002eb6c f   WdsService.obj
 0001:0002db9c       ?SetGetPacketServiceStatusIndicationCallbackCallback@WdsService@@QAAXP6AXPAXPAEG@Z0@Z 1002eb9c f   WdsService.obj
 0001:0002dbcc       ?Initialize@WdsService@@QAA_NPAUQMI_CHANNEL@@E@Z 1002ebcc f   WdsService.obj
 0001:0002dcec       ?Shutdown@WdsService@@QAAXXZ 1002ecec f   WdsService.obj
 0001:0002ddd0       ?ProcessSynchronousTransaction@WdsService@@QAAHPAVQmiTransaction@@GK@Z 1002edd0 f   WdsService.obj
 0001:0002e030       ?ProcessAsynchronousTransaction@WdsService@@QAAHPAVQmiTransaction@@GP6AXPAXPAEG@Z1@Z 1002f030 f   WdsService.obj
 0001:0002e1b4       ?HandleTransactionResponse@WdsService@@IAAXPAEG@Z 1002f1b4 f   WdsService.obj
 0001:0002e338       ?HandleTransactionIndication@WdsService@@IAAXPAEG@Z 1002f338 f   WdsService.obj
 0001:0002e434       ?ReadNotify@WdsService@@QAAXPAEG@Z 1002f434 f   WdsService.obj
 0001:0002e4b0       ?NewTransactionId@WdsService@@IAAGXZ 1002f4b0 f   WdsService.obj
 0001:0002e558       ?AddToOutstandingList@WdsService@@IAAXPAVQmiTransaction@@@Z 1002f558 f   WdsService.obj
 0001:0002e5dc       ?RemoveFromOutstandingList@WdsService@@IAAXPAVQmiTransaction@@@Z 1002f5dc f   WdsService.obj
 0001:0002e648       ?AddToFreeList@WdsService@@QAAXPAVQmiTransaction@@@Z 1002f648 f   WdsService.obj
 0001:0002e6cc       ?RemoveFromFreeList@WdsService@@IAAXPAVQmiTransaction@@@Z 1002f6cc f   WdsService.obj
 0001:0002e738       ?GetFromFreeList@WdsService@@QAAPAVQmiTransaction@@XZ 1002f738 f   WdsService.obj
 0001:0002e7a4       ??_EWdsService@@UAAPAXI@Z  1002f7a4 f i WdsService.obj
 0001:0002e7a4       ??_GWdsService@@UAAPAXI@Z  1002f7a4 f i WdsService.obj
 0001:0002e7e4       ?WrpHalt@@YAXPAX@Z         1002f7e4 f   wrp.obj
 0001:0002e9d0       ?WrpInitialize@@YAHPAHPAIPAW4_NDIS_MEDIUM@@IPAX3@Z 1002f9d0 f   wrp.obj
 0001:0002f090       ?DriverEntry@@YAJPAU_CEDRIVER_OBJECT@@PAU_UNICODE_STRING@@@Z 10030090 f   wrp.obj
 0001:0002f284       ?WrpSleep@@YAXK@Z          10030284 f   wrp.obj
 0001:0002f29c       ?WrpSend@@YAHPAXPAU_NDIS_PACKET@@I@Z 1003029c f   wrpcard.obj
 0001:0002f37c       ?WrpIndicateReceive@@YAXPAUsAdapterConfig@@PAEI@Z 1003037c f   wrpcard.obj
 0001:0002f540       ?WrpTransferData@@YAHPAU_NDIS_PACKET@@PAIPAX2II@Z 10030540 f   wrpcard.obj
 0001:0002f89c       ?WrpCheckForHang@@YAEPAX@Z 1003089c f   wrpcard.obj
 0001:0002f91c       ?WrpReset@@YAHPAEPAX@Z     1003091c f   wrpcard.obj
 0001:0002f998       ?WrpShutDown@@YAXPAX@Z     10030998 f   wrpcard.obj
 0001:0002f9d0       ?WrpPnPEventNotify@@YAXPAXW4_NDIS_DEVICE_PNP_EVENT@@0K@Z 100309d0 f   wrpcard.obj
 0001:0002fae4       ?WrpBuildLinearEthPacket@@YAEPAU_NDIS_PACKET@@PAEPAI@Z 10030ae4 f   wrpcard.obj
 0001:0002fc98       ?WrpIndicateSendComplete@@YAXPAUsAdapterConfig@@PAU_NDIS_PACKET@@E@Z 10030c98 f   wrpcard.obj
 0001:0002fde0       ?WrpQmiInitialize@@YAEPAUsAdapterConfig@@@Z 10030de0 f   wrpcard.obj
 0001:00030038       ?WrpQmiShutdown@@YAXPAUsAdapterConfig@@@Z 10031038 f   wrpcard.obj
 0001:00030078       ?WrpWdsSetEventReportResp@@YAXPAXPAEG@Z 10031078 f   wrpcard.obj
 0001:00030144       ?WrpWdsEventReportInd@@YAXPAXPAEG@Z 10031144 f   wrpcard.obj
 0001:00030870       ?WrpWdsGetPacketServiceStatusInd@@YAXPAXPAEG@Z 10031870 f   wrpcard.obj
 0001:00030bc0       ?WrpReconfigTimerDpc@@YAXPAX000@Z 10031bc0 f   wrpcard.obj
 0001:00030cdc       ?WrpResetPacketCount@@YAXPAUsAdapterConfig@@@Z 10031cdc f   wrpcard.obj
 0001:00030da8       ?WrpInitDriverBlock@@YAXXZ 10031da8 f   wrpdata.obj
 0001:00030e60       ?WrpGetDriverBlock@@YAPAUDRIVER_BLOCK@@XZ 10031e60 f   wrpdata.obj
 0001:00030e7c       ?WrpSetAdapterPointer@@YAXPAUsAdapterConfig@@@Z 10031e7c f   wrpdata.obj
 0001:00030ebc       ?WrpGetAdapterPointer@@YAPAUsAdapterConfig@@XZ 10031ebc f   wrpdata.obj
 0001:00030f00       ?WrpSetCardCount@@YAXE@Z   10031f00 f   wrpdata.obj
 0001:00030f40       ?WrpGetAdapterList@@YAPAU_LIST_ENTRY@@XZ 10031f40 f   wrpdata.obj
 0001:00030f60       ?WrpAcquireDriverSpinLock@@YAXXZ 10031f60 f   wrpdata.obj
 0001:00030f78       ?WrpReleaseDriverSpinLock@@YAXXZ 10031f78 f   wrpdata.obj
 0001:00030f90       ?WrpIncCardCount@@YAXXZ    10031f90 f   wrpdata.obj
 0001:00030fd0       ?WrpDecCardCount@@YAXXZ    10031fd0 f   wrpdata.obj
 0001:00031010       ?WrpGetCardCount@@YAKXZ    10032010 f   wrpdata.obj
 0001:00031054       ?WrpSetVendorDesc@@YAXPAUsAdapterConfig@@PAD@Z 10032054 f   wrpdata.obj
 0001:000310f0       ?WrpGetVendorDesc@@YAPADPAUsAdapterConfig@@@Z 100320f0 f   wrpdata.obj
 0001:00031138       ?WrpSetStartup@@YAXPAUsAdapterConfig@@E@Z 10032138 f   wrpdata.obj
 0001:00031178       ?WrpGetStartup@@YAEPAUsAdapterConfig@@@Z 10032178 f   wrpdata.obj
 0001:000311c4       ?WrpSetReset@@YAXPAUsAdapterConfig@@E@Z 100321c4 f   wrpdata.obj
 0001:000311e4       ?WrpGetReset@@YAEPAUsAdapterConfig@@@Z 100321e4 f   wrpdata.obj
 0001:00031230       ?WrpSetTestGateway@@YAXPAUsAdapterConfig@@E@Z 10032230 f   wrpdata.obj
 0001:00031270       ?WrpGetTestGateway@@YAEPAUsAdapterConfig@@@Z 10032270 f   wrpdata.obj
 0001:000312bc       ?WrpSetShutdownPolicy@@YAXPAUsAdapterConfig@@E@Z 100322bc f   wrpdata.obj
 0001:000312fc       ?WrpGetShutdownPolicy@@YAEPAUsAdapterConfig@@@Z 100322fc f   wrpdata.obj
 0001:00031348       ?WrpSetProductType@@YAXPAUsAdapterConfig@@G@Z 10032348 f   wrpdata.obj
 0001:00031388       ?WrpGetProductType@@YAGPAUsAdapterConfig@@@Z 10032388 f   wrpdata.obj
 0001:000313d4       ?WrpSetEnableWins@@YAXPAUsAdapterConfig@@E@Z 100323d4 f   wrpdata.obj
 0001:00031414       ?WrpGetEnableWins@@YAEPAUsAdapterConfig@@@Z 10032414 f   wrpdata.obj
 0001:00031460       ?WrpSetEnableWinsTemp@@YAXPAUsAdapterConfig@@E@Z 10032460 f   wrpdata.obj
 0001:000314a0       ?WrpGetEnableWinsTemp@@YAEPAUsAdapterConfig@@@Z 100324a0 f   wrpdata.obj
 0001:000314ec       ?WrpSetEnableTxTimer@@YAXPAUsAdapterConfig@@E@Z 100324ec f   wrpdata.obj
 0001:0003152c       ?WrpGetEnableTxTimer@@YAEPAUsAdapterConfig@@@Z 1003252c f   wrpdata.obj
 0001:00031578       ?WrpSetEnableDeepSleep@@YAXPAUsAdapterConfig@@E@Z 10032578 f   wrpdata.obj
 0001:000315b8       ?WrpGetEnableDeepSleep@@YAEPAUsAdapterConfig@@@Z 100325b8 f   wrpdata.obj
 0001:00031604       ?WrpAllocateMemory@@YAHPAUsAdapterConfig@@PAPAXIPBD@Z 10032604 f   wrpmemory.obj
 0001:00031698       ?WrpFreeMemory@@YAXPAUsAdapterConfig@@PAXIPBD@Z 10032698 f   wrpmemory.obj
 0001:00031718       ?OidToNameStr@@YAPADK@Z    10032718 f   wrpoid.obj
 0001:000320c8       ?WrpQueryInfo@@YAHPAXK0KPAK1@Z 100330c8 f   wrpoid.obj
 0001:000335e4       ?WrpSetInfo@@YAHPAXK0KPAK1@Z 100345e4 f   wrpoid.obj
 0001:00033c68       ?piput16_host_noinc@@YAXGPAPAE@Z 10034c68 f i wrpoid.obj
 0001:00033cc8       ?piput16_host@@YAXGPAPAE@Z 10034cc8 f i wrpoid.obj
 0001:00033d34       ?piput32_host_noinc@@YAXKPAPAEI@Z 10034d34 f i wrpoid.obj
 0001:00033ddc       ?piput64_host_noinc@@YAX_KPAPAEI@Z 10034ddc f i wrpoid.obj
 0001:00033f24       ?piputmulti_noinc@@YAXPAEPAPAEG@Z 10034f24 f i wrpoid.obj
 0001:00033f9c       ?piget16_host@@YAGPAPAE@Z  10034f9c f i wrpoid.obj
 0001:0003401c       ?piget32_host_noinc@@YAKPAPAE@Z 1003501c f i wrpoid.obj
 0001:000340d8       ?OpenRegistry@@YAXPAHPAPAX1@Z 100350d8 f   wrpregistry.obj
 0001:00034138       ?CloseRegistry@@YAXPAPAX@Z 10035138 f   wrpregistry.obj
 0001:00034184       ?ReadRegistry@@YAXPAHPAPAU_NDIS_CONFIGURATION_PARAMETER@@PAPAXPAU_UNICODE_STRING@@W4_NDIS_PARAMETER_TYPE@@@Z 10035184 f   wrpregistry.obj
 0001:000341dc       ?ConvertRegistryData@@YAEPAU_NDIS_CONFIGURATION_PARAMETER@@PADJ@Z 100351dc f   wrpregistry.obj
 0001:00034290       ?ConvertMacAddress@@YAEPAU_NDIS_CONFIGURATION_PARAMETER@@PAE@Z 10035290 f   wrpregistry.obj
 0001:00034500       NdisReleaseSpinLock        10035500 f   ndis:NDIS.dll
 0001:00034510       NdisAcquireSpinLock        10035510 f   ndis:NDIS.dll
 0001:00034520       NdisResetEvent             10035520 f   ndis:NDIS.dll
 0001:00034530       NdisSetEvent               10035530 f   ndis:NDIS.dll
 0001:00034540       NdisDeregisterAdapter      10035540 f   ndis:NDIS.dll
 0001:00034550       NdisRegisterAdapter        10035550 f   ndis:NDIS.dll
 0001:00034560       NdisMSleep                 10035560 f   ndis:NDIS.dll
 0001:00034570       NdisFreeSpinLock           10035570 f   ndis:NDIS.dll
 0001:00034580       NdisFreeEvent              10035580 f   ndis:NDIS.dll
 0001:00034590       NdisWaitEvent              10035590 f   ndis:NDIS.dll
 0001:000345a0       NdisCancelTimer            100355a0 f   ndis:NDIS.dll
 0001:000345b0       NdisMDeregisterAdapterShutdownHandler 100355b0 f   ndis:NDIS.dll
 0001:000345c0       NdisInitializeTimer        100355c0 f   ndis:NDIS.dll
 0001:000345d0       NdisInitializeEvent        100355d0 f   ndis:NDIS.dll
 0001:000345e0       NdisAllocateSpinLock       100355e0 f   ndis:NDIS.dll
 0001:000345f0       NdisWriteErrorLogEntry     100355f0 f   ndis:NDIS.dll
 0001:00034600       NdisMSetAttributesEx       10035600 f   ndis:NDIS.dll
 0001:00034610       NdisMRegisterAdapterShutdownHandler 10035610 f   ndis:NDIS.dll
 0001:00034620       NdisTerminateWrapper       10035620 f   ndis:NDIS.dll
 0001:00034630       NdisMRegisterMiniport      10035630 f   ndis:NDIS.dll
 0001:00034640       NdisInitializeWrapper      10035640 f   ndis:NDIS.dll
 0001:00034650       NdisQueryPacket            10035650 f   ndis:NDIS.dll
 0001:00034660       NdisSetTimer               10035660 f   ndis:NDIS.dll
 0001:00034670       NdisAllocateMemoryWithTag  10035670 f   ndis:NDIS.dll
 0001:00034680       NdisFreeMemory             10035680 f   ndis:NDIS.dll
 0001:00034690       NdisOpenConfiguration      10035690 f   ndis:NDIS.dll
 0001:000346a0       NdisCloseConfiguration     100356a0 f   ndis:NDIS.dll
 0001:000346b0       NdisReadConfiguration      100356b0 f   ndis:NDIS.dll
 0001:000346c0       NdisUnicodeStringToAnsiString 100356c0 f   ndis:NDIS.dll
 0001:000346d0       htons                      100356d0 f   ws2:WS2.dll
 0001:000346e0       htonl                      100356e0 f   ws2:WS2.dll
 0001:000346f0       CeSetThreadPriority        100356f0 f   coredll:COREDLL.dll
 0001:00034700       NKDbgPrintfW               10035700 f   coredll:COREDLL.dll
 0001:00034710       GetLastError               10035710 f   coredll:COREDLL.dll
 0001:00034720       RequestPowerNotifications  10035720 f   coredll:COREDLL.dll
 0001:00034730       CreateMsgQueue             10035730 f   coredll:COREDLL.dll
 0001:00034740       InitializeCriticalSection  10035740 f   coredll:COREDLL.dll
 0001:00034750       CreateThread               10035750 f   coredll:COREDLL.dll
 0001:00034760       CreateEventW               10035760 f   coredll:COREDLL.dll
 0001:00034770       CloseMsgQueue              10035770 f   coredll:COREDLL.dll
 0001:00034780       DeleteCriticalSection      10035780 f   coredll:COREDLL.dll
 0001:00034790       LeaveCriticalSection       10035790 f   coredll:COREDLL.dll
 0001:000347a0       CloseHandle                100357a0 f   coredll:COREDLL.dll
 0001:000347b0       WaitForSingleObject        100357b0 f   coredll:COREDLL.dll
 0001:000347c0       EnterCriticalSection       100357c0 f   coredll:COREDLL.dll
 0001:000347d0       EventModify                100357d0 f   coredll:COREDLL.dll
 0001:000347e0       Sleep                      100357e0 f   coredll:COREDLL.dll
 0001:000347f0       GetTickCount               100357f0 f   coredll:COREDLL.dll
 0001:00034800       WaitForMultipleObjects     10035800 f   coredll:COREDLL.dll
 0001:00034810       __rt_udiv                  10035810 f   coredll:COREDLL.dll
 0001:00034820       ReadMsgQueue               10035820 f   coredll:COREDLL.dll
 0001:00034830       memset                     10035830 f   coredll:COREDLL.dll
 0001:00034840       memcpy                     10035840 f   coredll:COREDLL.dll
 0001:00034850       vswprintf                  10035850 f   coredll:COREDLL.dll
 0001:00034860       ??3@YAXPAX@Z               10035860 f   coredll:COREDLL.dll
 0001:00034870       SetCommMask                10035870 f   coredll:COREDLL.dll
 0001:00034880       SetCommState               10035880 f   coredll:COREDLL.dll
 0001:00034890       CreateFileW                10035890 f   coredll:COREDLL.dll
 0001:000348a0       swprintf                   100358a0 f   coredll:COREDLL.dll
 0001:000348b0       ??2@YAPAXI@Z               100358b0 f   coredll:COREDLL.dll
 0001:000348c0       GetCommModemStatus         100358c0 f   coredll:COREDLL.dll
 0001:000348d0       EscapeCommFunction         100358d0 f   coredll:COREDLL.dll
 0001:000348e0       ReadFile                   100358e0 f   coredll:COREDLL.dll
 0001:000348f0       SetLastError               100358f0 f   coredll:COREDLL.dll
 0001:00034900       WriteFile                  10035900 f   coredll:COREDLL.dll
 0001:00034910       DeviceIoControl            10035910 f   coredll:COREDLL.dll
 0001:00034920       ??_L@YAXPAXIHP6AX0@Z1@Z    10035920 f   coredll:COREDLL.dll
 0001:00034930       ??_M@YAXPAXIHP6AX0@Z@Z     10035930 f   coredll:COREDLL.dll
 0001:00034940       strlen                     10035940 f   coredll:COREDLL.dll
 0001:00034950       OutputDebugStringW         10035950 f   coredll:COREDLL.dll
 0001:00034960       vsprintf                   10035960 f   coredll:COREDLL.dll
 0001:00034970       SystemTimeToFileTime       10035970 f   coredll:COREDLL.dll
 0001:00034980       GetSystemTime              10035980 f   coredll:COREDLL.dll
 0001:00034990       __rt_sdiv                  10035990 f   coredll:COREDLL.dll
 0001:000349a0       __rt_udiv64by64            100359a0 f   coredll:COREDLL.dll
 0001:000349b0       FlushFileBuffers           100359b0 f   coredll:COREDLL.dll
 0001:000349c0       SetFilePointer             100359c0 f   coredll:COREDLL.dll
 0001:000349d0       wcslen                     100359d0 f   coredll:COREDLL.dll
 0001:000349e0       RegCloseKey                100359e0 f   coredll:COREDLL.dll
 0001:000349f0       RegDeleteValueW            100359f0 f   coredll:COREDLL.dll
 0001:00034a00       RegOpenKeyExW              10035a00 f   coredll:COREDLL.dll
 0001:00034a10       wsprintfW                  10035a10 f   coredll:COREDLL.dll
 0001:00034a20       strncpy                    10035a20 f   coredll:COREDLL.dll
 0001:00034a30       InterlockedExchange        10035a30 f   coredll:COREDLL.dll
 0001:00034a40       __C_specific_handler       10035a40 f   coredll:COREDLL.dll
 0001:00034a50       LocalAllocTrace            10035a50 f   coredll:COREDLL.dll
 0001:00034a60       LocalFree                  10035a60 f   coredll:COREDLL.dll
 0001:00034a70       RegQueryValueExW           10035a70 f   coredll:COREDLL.dll
 0001:00034a80       RegSetValueExW             10035a80 f   coredll:COREDLL.dll
 0001:00034a90       RegCreateKeyExW            10035a90 f   coredll:COREDLL.dll
 0001:00034aa0       RegisterDbgZones           10035aa0 f   coredll:COREDLL.dll
 0001:00034ab0       wcscat                     10035ab0 f   coredll:COREDLL.dll
 0001:00034ac0       wcsncat                    10035ac0 f   coredll:COREDLL.dll
 0001:00034ad0       _snwprintf                 10035ad0 f   coredll:COREDLL.dll
 0001:00034ae0       rand                       10035ae0 f   coredll:COREDLL.dll
 0001:00034af0       FindClose                  10035af0 f   coredll:COREDLL.dll
 0001:00034b00       FindFirstFileW             10035b00 f   coredll:COREDLL.dll
 0001:00034b10       _wcsicmp                   10035b10 f   coredll:COREDLL.dll
 0001:00034b20       GetStoreInformation        10035b20 f   coredll:COREDLL.dll
 0001:00034b30       GlobalMemoryStatus         10035b30 f   coredll:COREDLL.dll
 0001:00034b40       HeapAllocTrace             10035b40 f   coredll:COREDLL.dll
 0001:00034b50       GetProcessHeap             10035b50 f   coredll:COREDLL.dll
 0001:00034b60       VirtualAlloc               10035b60 f   coredll:COREDLL.dll
 0001:00034b70       HeapFree                   10035b70 f   coredll:COREDLL.dll
 0001:00034b80       VirtualFree                10035b80 f   coredll:COREDLL.dll
 0001:00034b90       IsBadReadPtr               10035b90 f   coredll:COREDLL.dll
 0001:00034ba0       strcpy                     10035ba0 f   coredll:COREDLL.dll
 0001:00034bb0       TerminateThread            10035bb0 f   coredll:COREDLL.dll
 0001:00034bc0       StringCchPrintfW           10035bc0 f   coredll:COREDLL.dll
 0001:00034bd0       StringCchCatW              10035bd0 f   coredll:COREDLL.dll
 0001:00034be0       DeactivateDevice           10035be0 f   coredll:COREDLL.dll
 0001:00034bf0       wcscpy                     10035bf0 f   coredll:COREDLL.dll
 0001:00034c00       ActivateDeviceEx           10035c00 f   coredll:COREDLL.dll
 0001:00034c10       wcscmp                     10035c10 f   coredll:COREDLL.dll
 0001:00034c20       SystemParametersInfoW      10035c20 f   coredll:COREDLL.dll
 0001:00034c30       memcmp                     10035c30 f   coredll:COREDLL.dll
 0001:00034c40       MultiByteToWideChar        10035c40 f   coredll:COREDLL.dll
 0001:00034c50       SetSystemPowerState        10035c50 f   coredll:COREDLL.dll
 0001:00034c60       wcsstr                     10035c60 f   coredll:COREDLL.dll
 0001:00034c70       _wcslwr                    10035c70 f   coredll:COREDLL.dll
 0001:00034c80       GetSystemPowerState        10035c80 f   coredll:COREDLL.dll
 0001:00034c90       sprintf                    10035c90 f   coredll:COREDLL.dll
 0001:00034ca0       _DllMainCRTStartup         10035ca0 f   corelibc:pegdmain.obj
 0001:00034d38       __security_check_cookie    10035d38     corelibc:armsecgs.obj
 0001:00034d4c       __gsfailure                10035d4c     corelibc:armsecgs.obj
 0001:00034d90       _onexit                    10035d90 f   corelibc:onexit.obj
 0001:00034e3c       atexit                     10035e3c f   corelibc:onexit.obj
 0001:00034e5c       GetCurrentProcess          10035e5c f i corelibc:crt0dat.obj
 0001:00034e98       _cinit                     10035e98 f   corelibc:crt0dat.obj
 0001:00035008       exit                       10036008 f   corelibc:crt0dat.obj
 0001:00035020       _exit                      10036020 f   corelibc:crt0dat.obj
 0001:00035038       _cexit                     10036038 f   corelibc:crt0dat.obj
 0001:00035054       _c_exit                    10036054 f   corelibc:crt0dat.obj
 0001:000350a0       __security_init_cookie     100360a0 f   corelibc:seccinit.obj
 0001:000350f0       __GSHandlerCheckCommon     100360f0 f   LIBCMTD:gshandler.obj
 0001:00035138       __GSHandlerCheck           10036138 f   LIBCMTD:gshandler.obj
 0001:00035168       __InternalCxxFrameHandler  10036168 f   LIBCMTD:frame_ce.obj
 0001:00035344       __CxxFrameHandler3         10036344 f   LIBCMTD:frame_ce.obj
 0001:00035b20       __FrameUnwindToState       10036b20 f   LIBCMTD:frame_ce.obj
 0001:000368cc       ?_DestructExceptionObject@@YAXPAUEHExceptionRecord@@E@Z 100378cc f   LIBCMTD:frame_ce.obj
 0001:00036a1c       ?_OffsetToAddress@@YAPAXHPAKK@Z 10037a1c f   LIBCMTD:frame_ce.obj
 0001:00036aa8       ?FindFrameInfo@@YAPAU_FrameInfo@@PAK@Z 10037aa8 f   LIBCMTD:frame_ce.obj
 0001:00036b30       ?FindCatchFrameInfo@@YAPAU_FrameInfo@@PAK@Z 10037b30 f   LIBCMTD:frame_ce.obj
 0001:00036bb4       ?_GetRangeOfTrysToCheck@@YAPBU_s_TryBlockMapEntry@@PBU_s_FuncInfo@@HHPAI1@Z 10037bb4 f   LIBCMTD:frame_ce.obj
 0001:00036cac       __GSHandlerCheck_EH        10037cac f   LIBCMTD:gshandlereh.obj
 0001:00036d40       __GSHandlerCheck_SEH       10037d40 f   LIBCMTD:gshandlerseh.obj
 0001:00036da8       GetCRTStorage              10037da8 f   LIBCMTD:corecrt.obj
 0001:00036eb8       TlsAlloc                   10037eb8 f i LIBCMTD:corecrt.obj
 0001:00036ef4       TlsFree                    10037ef4 f i LIBCMTD:corecrt.obj
 0001:00036f38       ?FindFrameForUnwind@@YAPAKPAKPBU_s_FuncInfo@@@Z 10037f38 f   LIBCMTD:mdframe_arm.obj
 0001:00036fd0       ?FindCatchFrame@@YAPAKPAKK@Z 10037fd0 f   LIBCMTD:mdframe_arm.obj
 0001:00037068       ?AdjustFrameForCatch@@YAPAKPAKPBU_s_FuncInfo@@@Z 10038068 f   LIBCMTD:mdframe_arm.obj
 0001:00037108       ?GetCurrentState@@YAHPAKPAU_DISPATCHER_CONTEXT@@PBU_s_FuncInfo@@@Z 10038108 f   LIBCMTD:ehstate_arm_mips.obj
 0001:000371e4       _CallSettingFrame          100381e4     LIBCMTD:handlers_arm.obj
 0001:00037228       __report_gsfailure         10038228 f   coredll:COREDLL.dll
 0001:00037238       LocalReAlloc               10038238 f   coredll:COREDLL.dll
 0001:00037248       LocalAlloc                 10038248 f   coredll:COREDLL.dll
 0001:00037258       LocalSize                  10038258 f   coredll:COREDLL.dll
 0001:00037268       __security_gen_cookie      10038268 f   coredll:COREDLL.dll
 0001:00037278       strcmp                     10038278 f   coredll:COREDLL.dll
 0001:00037288       ?terminate@std@@YAXXZ      10038288 f   coredll:COREDLL.dll
 0001:00037298       memmove                    10038298 f   coredll:COREDLL.dll
 0001:000372a8       TlsSetValue                100382a8 f   coredll:COREDLL.dll
 0001:000372b8       TlsGetValue                100382b8 f   coredll:COREDLL.dll
 0001:000372c8       InterlockedCompareExchange 100382c8 f   coredll:COREDLL.dll
 0001:000372d8       TlsCall                    100382d8 f   coredll:COREDLL.dll
 0002:00003420       ??_C@_15JNBOKNOG@?$AA?$AN?$AA?6?$AA?$AA@ 1003c420     commdevice.obj
 0002:00003428       ??_7CommDevice@@6B@        1003c428     commdevice.obj
 0002:00003968       ??_7CtlService@@6B@        1003c968     CtlService.obj
 0002:0000396c       ??_7DmsService@@6B@        1003c96c     DmsService.obj
 0002:000075e0       ??_7RilOutContextPool@@6B@ 100405e0     RilOutContextPool.obj
 0002:00007740       ??_7RilPacketPool@@6B@     10040740     RilPacketPool.obj
 0002:0001ff3c       ??_7WdsService@@6B@        10058f3c     WdsService.obj
 0002:00021d70       __IMPORT_DESCRIPTOR_NDIS   1005ad70     ndis:NDIS.dll
 0002:00021d84       __IMPORT_DESCRIPTOR_WS2    1005ad84     ws2:WS2.dll
 0002:00021d98       __IMPORT_DESCRIPTOR_COREDLL 1005ad98     coredll:COREDLL.dll
 0002:00021dac       __NULL_IMPORT_DESCRIPTOR   1005adac     ndis:NDIS.dll
 0003:00000000       __imp_??_L@YAXPAXIHP6AX0@Z1@Z 1005c000     coredll:COREDLL.dll
 0003:00000004       __imp_InterlockedCompareExchange 1005c004     coredll:COREDLL.dll
 0003:00000008       __imp_TlsGetValue          1005c008     coredll:COREDLL.dll
 0003:0000000c       __imp_TlsSetValue          1005c00c     coredll:COREDLL.dll
 0003:00000010       __imp_memmove              1005c010     coredll:COREDLL.dll
 0003:00000014       __imp_?terminate@std@@YAXXZ 1005c014     coredll:COREDLL.dll
 0003:00000018       __imp_strcmp               1005c018     coredll:COREDLL.dll
 0003:0000001c       __imp___security_gen_cookie 1005c01c     coredll:COREDLL.dll
 0003:00000020       __imp_LocalSize            1005c020     coredll:COREDLL.dll
 0003:00000024       __imp_LocalAlloc           1005c024     coredll:COREDLL.dll
 0003:00000028       __imp_LocalReAlloc         1005c028     coredll:COREDLL.dll
 0003:0000002c       __imp___report_gsfailure   1005c02c     coredll:COREDLL.dll
 0003:00000030       __imp_sprintf              1005c030     coredll:COREDLL.dll
 0003:00000034       __imp_GetSystemPowerState  1005c034     coredll:COREDLL.dll
 0003:00000038       __imp__wcslwr              1005c038     coredll:COREDLL.dll
 0003:0000003c       __imp_wcsstr               1005c03c     coredll:COREDLL.dll
 0003:00000040       __imp_SetSystemPowerState  1005c040     coredll:COREDLL.dll
 0003:00000044       __imp_MultiByteToWideChar  1005c044     coredll:COREDLL.dll
 0003:00000048       __imp_memcmp               1005c048     coredll:COREDLL.dll
 0003:0000004c       __imp_SystemParametersInfoW 1005c04c     coredll:COREDLL.dll
 0003:00000050       __imp_wcscmp               1005c050     coredll:COREDLL.dll
 0003:00000054       __imp_ActivateDeviceEx     1005c054     coredll:COREDLL.dll
 0003:00000058       __imp_wcscpy               1005c058     coredll:COREDLL.dll
 0003:0000005c       __imp_DeactivateDevice     1005c05c     coredll:COREDLL.dll
 0003:00000060       __imp_StringCchCatW        1005c060     coredll:COREDLL.dll
 0003:00000064       __imp_StringCchPrintfW     1005c064     coredll:COREDLL.dll
 0003:00000068       __imp_TerminateThread      1005c068     coredll:COREDLL.dll
 0003:0000006c       __imp_strcpy               1005c06c     coredll:COREDLL.dll
 0003:00000070       __imp_IsBadReadPtr         1005c070     coredll:COREDLL.dll
 0003:00000074       __imp_VirtualFree          1005c074     coredll:COREDLL.dll
 0003:00000078       __imp_HeapFree             1005c078     coredll:COREDLL.dll
 0003:0000007c       __imp_VirtualAlloc         1005c07c     coredll:COREDLL.dll
 0003:00000080       __imp_CeSetThreadPriority  1005c080     coredll:COREDLL.dll
 0003:00000084       __imp_NKDbgPrintfW         1005c084     coredll:COREDLL.dll
 0003:00000088       __imp_GetLastError         1005c088     coredll:COREDLL.dll
 0003:0000008c       __imp_RequestPowerNotifications 1005c08c     coredll:COREDLL.dll
 0003:00000090       __imp_CreateMsgQueue       1005c090     coredll:COREDLL.dll
 0003:00000094       __imp_InitializeCriticalSection 1005c094     coredll:COREDLL.dll
 0003:00000098       __imp_CreateThread         1005c098     coredll:COREDLL.dll
 0003:0000009c       __imp_CreateEventW         1005c09c     coredll:COREDLL.dll
 0003:000000a0       __imp_CloseMsgQueue        1005c0a0     coredll:COREDLL.dll
 0003:000000a4       __imp_DeleteCriticalSection 1005c0a4     coredll:COREDLL.dll
 0003:000000a8       __imp_LeaveCriticalSection 1005c0a8     coredll:COREDLL.dll
 0003:000000ac       __imp_CloseHandle          1005c0ac     coredll:COREDLL.dll
 0003:000000b0       __imp_WaitForSingleObject  1005c0b0     coredll:COREDLL.dll
 0003:000000b4       __imp_EnterCriticalSection 1005c0b4     coredll:COREDLL.dll
 0003:000000b8       __imp_EventModify          1005c0b8     coredll:COREDLL.dll
 0003:000000bc       __imp_Sleep                1005c0bc     coredll:COREDLL.dll
 0003:000000c0       __imp_GetTickCount         1005c0c0     coredll:COREDLL.dll
 0003:000000c4       __imp_WaitForMultipleObjects 1005c0c4     coredll:COREDLL.dll
 0003:000000c8       __imp___rt_udiv            1005c0c8     coredll:COREDLL.dll
 0003:000000cc       __imp_ReadMsgQueue         1005c0cc     coredll:COREDLL.dll
 0003:000000d0       __imp_memset               1005c0d0     coredll:COREDLL.dll
 0003:000000d4       __imp_memcpy               1005c0d4     coredll:COREDLL.dll
 0003:000000d8       __imp_vswprintf            1005c0d8     coredll:COREDLL.dll
 0003:000000dc       __imp_??3@YAXPAX@Z         1005c0dc     coredll:COREDLL.dll
 0003:000000e0       __imp_SetCommMask          1005c0e0     coredll:COREDLL.dll
 0003:000000e4       __imp_SetCommState         1005c0e4     coredll:COREDLL.dll
 0003:000000e8       __imp_CreateFileW          1005c0e8     coredll:COREDLL.dll
 0003:000000ec       __imp_swprintf             1005c0ec     coredll:COREDLL.dll
 0003:000000f0       __imp_??2@YAPAXI@Z         1005c0f0     coredll:COREDLL.dll
 0003:000000f4       __imp_GetCommModemStatus   1005c0f4     coredll:COREDLL.dll
 0003:000000f8       __imp_EscapeCommFunction   1005c0f8     coredll:COREDLL.dll
 0003:000000fc       __imp_ReadFile             1005c0fc     coredll:COREDLL.dll
 0003:00000100       __imp_SetLastError         1005c100     coredll:COREDLL.dll
 0003:00000104       __imp_WriteFile            1005c104     coredll:COREDLL.dll
 0003:00000108       __imp_DeviceIoControl      1005c108     coredll:COREDLL.dll
 0003:0000010c       __imp_TlsCall              1005c10c     coredll:COREDLL.dll
 0003:00000110       __imp_??_M@YAXPAXIHP6AX0@Z@Z 1005c110     coredll:COREDLL.dll
 0003:00000114       __imp_strlen               1005c114     coredll:COREDLL.dll
 0003:00000118       __imp_OutputDebugStringW   1005c118     coredll:COREDLL.dll
 0003:0000011c       __imp_vsprintf             1005c11c     coredll:COREDLL.dll
 0003:00000120       __imp_SystemTimeToFileTime 1005c120     coredll:COREDLL.dll
 0003:00000124       __imp_GetSystemTime        1005c124     coredll:COREDLL.dll
 0003:00000128       __imp___rt_sdiv            1005c128     coredll:COREDLL.dll
 0003:0000012c       __imp___rt_udiv64by64      1005c12c     coredll:COREDLL.dll
 0003:00000130       __imp_FlushFileBuffers     1005c130     coredll:COREDLL.dll
 0003:00000134       __imp_SetFilePointer       1005c134     coredll:COREDLL.dll
 0003:00000138       __imp_wcslen               1005c138     coredll:COREDLL.dll
 0003:0000013c       __imp_RegCloseKey          1005c13c     coredll:COREDLL.dll
 0003:00000140       __imp_RegDeleteValueW      1005c140     coredll:COREDLL.dll
 0003:00000144       __imp_RegOpenKeyExW        1005c144     coredll:COREDLL.dll
 0003:00000148       __imp_wsprintfW            1005c148     coredll:COREDLL.dll
 0003:0000014c       __imp_strncpy              1005c14c     coredll:COREDLL.dll
 0003:00000150       __imp_InterlockedExchange  1005c150     coredll:COREDLL.dll
 0003:00000154       __imp___C_specific_handler 1005c154     coredll:COREDLL.dll
 0003:00000158       __imp_LocalAllocTrace      1005c158     coredll:COREDLL.dll
 0003:0000015c       __imp_LocalFree            1005c15c     coredll:COREDLL.dll
 0003:00000160       __imp_RegQueryValueExW     1005c160     coredll:COREDLL.dll
 0003:00000164       __imp_RegSetValueExW       1005c164     coredll:COREDLL.dll
 0003:00000168       __imp_RegCreateKeyExW      1005c168     coredll:COREDLL.dll
 0003:0000016c       __imp_RegisterDbgZones     1005c16c     coredll:COREDLL.dll
 0003:00000170       __imp_wcscat               1005c170     coredll:COREDLL.dll
 0003:00000174       __imp_wcsncat              1005c174     coredll:COREDLL.dll
 0003:00000178       __imp__snwprintf           1005c178     coredll:COREDLL.dll
 0003:0000017c       __imp_rand                 1005c17c     coredll:COREDLL.dll
 0003:00000180       __imp_FindClose            1005c180     coredll:COREDLL.dll
 0003:00000184       __imp_FindFirstFileW       1005c184     coredll:COREDLL.dll
 0003:00000188       __imp__wcsicmp             1005c188     coredll:COREDLL.dll
 0003:0000018c       __imp_GetStoreInformation  1005c18c     coredll:COREDLL.dll
 0003:00000190       __imp_GlobalMemoryStatus   1005c190     coredll:COREDLL.dll
 0003:00000194       __imp_HeapAllocTrace       1005c194     coredll:COREDLL.dll
 0003:00000198       __imp_GetProcessHeap       1005c198     coredll:COREDLL.dll
 0003:0000019c       \177COREDLL_NULL_THUNK_DATA 1005c19c     coredll:COREDLL.dll
 0003:000001a0       __imp_NdisMSetAttributesEx 1005c1a0     ndis:NDIS.dll
 0003:000001a4       __imp_NdisAcquireSpinLock  1005c1a4     ndis:NDIS.dll
 0003:000001a8       __imp_NdisResetEvent       1005c1a8     ndis:NDIS.dll
 0003:000001ac       __imp_NdisUnicodeStringToAnsiString 1005c1ac     ndis:NDIS.dll
 0003:000001b0       __imp_NdisReadConfiguration 1005c1b0     ndis:NDIS.dll
 0003:000001b4       __imp_NdisCloseConfiguration 1005c1b4     ndis:NDIS.dll
 0003:000001b8       __imp_NdisOpenConfiguration 1005c1b8     ndis:NDIS.dll
 0003:000001bc       __imp_NdisFreeMemory       1005c1bc     ndis:NDIS.dll
 0003:000001c0       __imp_NdisAllocateMemoryWithTag 1005c1c0     ndis:NDIS.dll
 0003:000001c4       __imp_NdisSetTimer         1005c1c4     ndis:NDIS.dll
 0003:000001c8       __imp_NdisQueryPacket      1005c1c8     ndis:NDIS.dll
 0003:000001cc       __imp_NdisInitializeWrapper 1005c1cc     ndis:NDIS.dll
 0003:000001d0       __imp_NdisMRegisterMiniport 1005c1d0     ndis:NDIS.dll
 0003:000001d4       __imp_NdisTerminateWrapper 1005c1d4     ndis:NDIS.dll
 0003:000001d8       __imp_NdisMRegisterAdapterShutdownHandler 1005c1d8     ndis:NDIS.dll
 0003:000001dc       __imp_NdisReleaseSpinLock  1005c1dc     ndis:NDIS.dll
 0003:000001e0       __imp_NdisWriteErrorLogEntry 1005c1e0     ndis:NDIS.dll
 0003:000001e4       __imp_NdisAllocateSpinLock 1005c1e4     ndis:NDIS.dll
 0003:000001e8       __imp_NdisInitializeEvent  1005c1e8     ndis:NDIS.dll
 0003:000001ec       __imp_NdisInitializeTimer  1005c1ec     ndis:NDIS.dll
 0003:000001f0       __imp_NdisMDeregisterAdapterShutdownHandler 1005c1f0     ndis:NDIS.dll
 0003:000001f4       __imp_NdisCancelTimer      1005c1f4     ndis:NDIS.dll
 0003:000001f8       __imp_NdisWaitEvent        1005c1f8     ndis:NDIS.dll
 0003:000001fc       __imp_NdisFreeEvent        1005c1fc     ndis:NDIS.dll
 0003:00000200       __imp_NdisFreeSpinLock     1005c200     ndis:NDIS.dll
 0003:00000204       __imp_NdisMSleep           1005c204     ndis:NDIS.dll
 0003:00000208       __imp_NdisRegisterAdapter  1005c208     ndis:NDIS.dll
 0003:0000020c       __imp_NdisDeregisterAdapter 1005c20c     ndis:NDIS.dll
 0003:00000210       __imp_NdisSetEvent         1005c210     ndis:NDIS.dll
 0003:00000214       \177NDIS_NULL_THUNK_DATA   1005c214     ndis:NDIS.dll
 0003:00000218       __imp_htonl                1005c218     ws2:WS2.dll
 0003:0000021c       __imp_htons                1005c21c     ws2:WS2.dll
 0003:00000220       \177WS2_NULL_THUNK_DATA    1005c220     ws2:WS2.dll
 0003:00000224       __xc_a                     1005c224     corelibc:crt0init.obj
 0003:00000230       __xc_z                     1005c230     corelibc:crt0init.obj
 0003:00000234       __xi_a                     1005c234     corelibc:crt0init.obj
 0003:00000238       __xi_z                     1005c238     corelibc:crt0init.obj
 0003:0000023c       __xp_a                     1005c23c     corelibc:crt0init.obj
 0003:00000240       __xp_z                     1005c240     corelibc:crt0init.obj
 0003:00000244       __xt_a                     1005c244     corelibc:crt0init.obj
 0003:00000248       __xt_z                     1005c248     corelibc:crt0init.obj
 0003:00000250       ?WceHandle@@3PAXA          1005c250     dpwce.obj
 0003:00000268       ?g_IsSavePowerInD2@@3HA    1005c268     swicom.obj
 0003:0000026c       ?gIsPowerManagedSupported@@3HA 1005c26c     swicom.obj
 0003:00000270       dpCurSettings              1005c270     swicom.obj
 0003:000006b4       ?InitCommandNames@@3PAPA_WA 1005c6b4     swiroutines.obj
 0003:000006d8       ?gdwResumeDetectInterval@@3KA 1005c6d8     swiusb.obj
 0003:000006dc       ?g_bFirstTime@@3HA         1005c6dc     swiusb.obj
 0003:000006e0       ?gArpResponseFrame@@3PAEA  1005c6e0     swiusb.obj
 0003:00000710       ?gDHCPDiscoveryFrame@@3PAEA 1005c710     swiusb.obj
 0003:00000868       ?gDHCPRequestFrame@@3PAEA  1005c868     swiusb.obj
 0003:000009c0       ?HighestAcceptableMax@@3T_LARGE_INTEGER@@A 1005c9c0     wrpdata.obj
 0003:000009c8       __security_cookie_complement 1005c9c8     corelibc:seccook.obj
 0003:000009cc       __security_cookie          1005c9cc     corelibc:seccook.obj
 0003:000009d8       ?g_dwLastDeviceResumedTickCount@@3KA 1005c9d8     CEPowerControl.obj
 0003:000021e0       ?gPrintCount@@3IA          1005e1e0     dpwce.obj
 0003:000021e8       ?gwszSWIUSBKey@@3PA_WA     1005e1e8     swicom.obj
 0003:000023e8       ?pOpenPortList@@3PAPAUVSP_OPEN_INFO@@A 1005e3e8     swicom.obj
 0003:00002408       ?CSDisplayRawData@@3UCRITICAL_SECTION@@A 1005e408     swicom.obj
 0003:0000241c       ?hDllInstance@@3PAXA       1005e41c     swicom.obj
 0003:00002420       ?guiCOMPortOpenCount@@3IA  1005e420     swicom.obj
 0003:00002424       ?gDevicePwrState@@3W4_CEDEVICE_POWER_STATE@@A 1005e424     swicom.obj
 0003:00002428       ?g_IsNMEAInProgress@@3HA   1005e428     swicom.obj
 0003:0000242c       ?gIsUseUnAttendedMode@@3HA 1005e42c     swicom.obj
 0003:00002430       ?bValidInstance@@3EA       1005e430     swicom.obj
 0003:00002434       ?alreadyAttached@@3HA      1005e434     swicom.obj
 0003:00002438       ?gMemoryCounter@@3KA       1005e438     swiroutines.obj
 0003:0000243c       ?gdwLastFreeSize@@3KA      1005e43c     swiroutines.obj
 0003:00002440       ?g_IsTerminalSuspended@@3HA 1005e440     swiusb.obj
 0003:00002444       ?gUseNdisConfiguration@@3KA 1005e444     swiusb.obj
 0003:00002448       ?CSUSBDeviceState@@3UCRITICAL_SECTION@@A 1005e448     swiusb.obj
 0003:0000245c       ?CSComPortOpenCount@@3UCRITICAL_SECTION@@A 1005e45c     swiusb.obj
 0003:00002470       ?CSSWIUsbMemoryControl@@3UCRITICAL_SECTION@@A 1005e470     swiusb.obj
 0003:00002484       ?bWindowsMobile@@3KA       1005e484     swiusb.obj
 0003:00002488       ?gTlpContext@@3UTLP_CONTEXT@@A 1005e488     swiusb.obj
 0003:00002a80       ?gdwIdleTimeout@@3KA       1005ea80     swiusb.obj
 0003:00002a84       ?gQmiFiltering@@3KA        1005ea84     swiusb.obj
 0003:00002a88       ?gQmiFilterCnt@@3KA        1005ea88     swiusb.obj
 0003:00002a8c       ?gQmiFilter@@3PAKA         1005ea8c     swiusb.obj
 0003:00002ac8       ?gdwDefaultTransferSize@@3KA 1005eac8     swiusb.obj
 0003:00002acc       ?dwThreadId@@3KA           1005eacc     swiusb.obj
 0003:00002ad0       ?hActivityThread@@3PAXA    1005ead0     swiusb.obj
 0003:00002ad4       ?gdwMaxAllocateSizePerChunk@@3KA 1005ead4     swiusb.obj
 0003:00002ad8       ?gEnableDataBundle@@3KA    1005ead8     swiusb.obj
 0003:00002adc       ?gDeviceRemoteWakeupReg@@3KA 1005eadc     swiusb.obj
 0003:00002ae0       ?ghDeviceInstalledEvent@@3PAXA 1005eae0     swiusb.obj
 0003:00002ae4       ?hDeviceCloseEvent@@3PAXA  1005eae4     swiusb.obj
 0003:00002ae8       ?hUSBResumeEvent@@3PAXA    1005eae8     swiusb.obj
 0003:00002aec       ?hUSBSuspendEvent@@3PAXA   1005eaec     swiusb.obj
 0003:00002af0       ?hUSBActivityEvent@@3PAXA  1005eaf0     swiusb.obj
 0003:00002af4       ?hHostJustResumedEvent@@3PAXA 1005eaf4     swiusb.obj
 0003:00002af8       ?hPortRemoteWakeup@@3PAXA  1005eaf8     swiusb.obj
 0003:00002afc       ?hSendArpResponseEvent@@3PAXA 1005eafc     swiusb.obj
 0003:00002b00       ?hSendDHCPDiscoveryEvent@@3PAXA 1005eb00     swiusb.obj
 0003:00002b04       ?hSendDHCPRequestEvent@@3PAXA 1005eb04     swiusb.obj
 0003:00002b08       ?g_IsRemoteWakeUpCallbackSupported@@3HA 1005eb08     swiusb.obj
 0003:00002b0c       ?ghModemPresent@@3PAXA     1005eb0c     swiusb.obj
 0003:00002b10       ?ghModemAbsent@@3PAXA      1005eb10     swiusb.obj
 0003:00002b14       ?gQmiCtlMsg@@3U_QMICTL_MSG@@A 1005eb14     swiusb.obj
 0003:00002b28       ?gModem@@3U_SW_MODEM@@A    1005eb28     swiusb.obj
 0003:00003660       __onexitend                1005f660     <common>
 0003:00003664       __onexitbegin              1005f664     <common>
 0003:00003668       _exitflag                  1005f668     <common>
 0003:0000366c       _pRawDllMain               1005f66c     <common>

 entry point at        0001:00034ca0

 Static symbols

 0001:000034c4       __unwind$38251             100044c4 f   commdevice.obj
 0001:000034e4       __unwind$38252             100044e4 f   commdevice.obj
 0001:00005234       __unwind$27620             10006234 f   commentry.obj
 0001:000070fc       ?dp_print_hex@@YAXPAEPBEH@Z 100080fc f   dpwce.obj
 0001:000071b4       ?dp_print_char@@YAXPAEPBEH@Z 100081b4 f   dpwce.obj
 0001:0000d3a8       ?QMIIOControl@@YAHPAUQMI_OPEN_INFO@@KPAEK1KPAK@Z 1000e3a8 f   qmicom.obj
 0001:0000d43c       ?NopIOControl@@YAHPAUQMI_OPEN_INFO@@KPAEK1KPAK@Z 1000e43c f   qmicom.obj
 0001:0000dca8       ?EventIOControl@@YAHPAUQMI_OPEN_INFO@@KPAEK1KPAK@Z 1000eca8 f   qmicom.obj
 0001:0000e20c       ?MdmIOControl@@YAHPAUQMI_OPEN_INFO@@KPAEK1KPAK@Z 1000f20c f   qmicom.obj
 0001:0000fdb8       __unwind$37965             10010db8 f   swdcom.obj
 0001:0000fdd0       __unwind$37966             10010dd0 f   swdcom.obj
 0001:00014cd8       ?ProcessExiting@@YAHPAUVSP_OPEN_INFO@@@Z 10015cd8 f   swicom.obj
 0001:00015ed8       ?NopIOControl@@YAHPAUVSP_OPEN_INFO@@KPAEK1KPAK@Z 10016ed8 f   swicom.obj
 0001:00016744       ?EventIOControl@@YAHPAUVSP_OPEN_INFO@@KPAEK1KPAK@Z 10017744 f   swicom.obj
 0001:00016ca8       ?MdmIOControl@@YAHPAUVSP_OPEN_INFO@@KPAEK1KPAK@Z 10017ca8 f   swicom.obj
 0001:000173d0       ?SWIUsbIOControl@@YAHPAUVSP_OPEN_INFO@@KPAEK1KPAK@Z 100183d0 f   swicom.obj
 0001:0001bf80       __unwind$40968             1001cf80 f   swiusb.obj
 0001:0001d63c       __unwind$41142             1001e63c f   swiusb.obj
 0001:0001d92c       __unwind$41190             1001e92c f   swiusb.obj
 0001:0001dfb8       ?BulkInDirectIpThread@@YAXPAPAX@Z 1001efb8 f   swiusb.obj
 0001:0001f9b0       ?BulkInDirectIpNoTlpThread@@YAXPAPAX@Z 100209b0 f   swiusb.obj
 0001:00021ba0       ?BulkOutDirectIpThread@@YAXPAPAX@Z 10022ba0 f   swiusb.obj
 0001:00022334       ?TransmitChannelBytesDirectIp@@YAHPAUSWD_CHANNEL@@PAEI@Z 10023334 f   swiusb.obj
 0001:000223f8       ?TransmitBytesDirectIp@@YAHPAUSWD_CHANNEL@@PAEI@Z 100233f8 f   swiusb.obj
 0001:00022b10       ?InterruptDirectIpThread@@YAXPAPAX@Z 10023b10 f   swiusb.obj
 0001:0002838c       ?BulkInThread@@YAXPAPAX@Z  1002938c f   swiusb.obj
 0001:00029e48       ?BulkOutThread@@YAXPAPAX@Z 1002ae48 f   swiusb.obj
 0001:0002a260       ?TransmitChannelBytes@@YAHPAUSW_CHANNEL@@PAEI@Z 1002b260 f   swiusb.obj
 0001:0002a324       ?TransmitBytes@@YAHPAUSW_CHANNEL@@PAEI@Z 1002b324 f   swiusb.obj
 0001:0002a84c       ?BulkOutMiniportThread@@YAXPAPAX@Z 1002b84c f   swiusb.obj
 0001:0002ae98       ?InterruptThread@@YAXPAPAX@Z 1002be98 f   swiusb.obj
 0001:0002ca84       ?ParseAndAddToReadQueue@@YAXPAEIPAUSW_CHANNEL@@@Z 1002da84 f   swiusb.obj
 0001:0002cb4c       ?ParseTlpTransfer@@YAXPAEIPAXP6AX0I1@Z@Z 1002db4c f   swiusb.obj
 0001:0002cea0       ?EthernetFrameHandlerMiniport@@YAXPAEIPAX@Z 1002dea0 f   swiusb.obj
 0001:0002ced8       ?ParseAndAddToRil@@YAXPAEIPAUSWD_CHANNEL@@@Z 1002ded8 f   swiusb.obj
 0001:0002cf2c       ?EthernetFrameHandlerRil@@YAXPAEIPAX@Z 1002df2c f   swiusb.obj
 0001:0002d238       ?EthernetFrameHandlerRilPacket@@YAXPAUSWD_CHANNEL@@PAPAUrilndispacket_tag@@@Z 1002e238 f   swiusb.obj
 0001:0002d7d0       ?ReleasePendingOutPackets@@YAXPAUSWD_CHANNEL@@@Z 1002e7d0 f   swiusb.obj
 0001:0002e95c       ?deregisterAdapter@@YAXPAUsAdapterConfig@@@Z 1002f95c f   wrp.obj
 0001:0002ee68       ?ReadConfigurationInfo@@YAHPAUsAdapterConfig@@PAX1PAE@Z 1002fe68 f   wrp.obj
 0001:0002efe4       ?registerAdapter@@YAHPAUsAdapterConfig@@@Z 1002ffe4 f   wrp.obj
 0001:00033340       ?OidFillOidList@@YAHPAEKPAK1@Z 10034340 f   wrpoid.obj
 0001:00033abc       ?SetPacketFilter@@YAHPAUsAdapterConfig@@K@Z 10034abc f   wrpoid.obj
 0001:00033b5c       ?SetMulticastList@@YAHPAUsAdapterConfig@@PAXKPAK2@Z 10034b5c f   wrpoid.obj
 0001:00034e64       _initterm                  10035e64 f   corelibc:crt0dat.obj
 0001:00034f04       doexit                     10035f04 f   corelibc:crt0dat.obj
 0001:000353c0       ?FindHandler@@YAEPAUEHExceptionRecord@@PAKPAU_CONTEXT@@PAU_DISPATCHER_CONTEXT@@PBU_s_FuncInfo@@H@Z 100363c0 f   LIBCMTD:frame_ce.obj
 0001:000359b4       ?TypeMatch@@YAHPBU_s_HandlerType@@PBU_s_CatchableType@@PBU_s_ThrowInfo@@@Z 100369b4 f   LIBCMTD:frame_ce.obj
 0001:00035d78       ?FrameUnwindFilter@@YAHPAU_EXCEPTION_POINTERS@@@Z 10036d78 f   LIBCMTD:frame_ce.obj
 0001:00035e04       ?CallCatchBlock@@YAPAXPAUEHExceptionRecord@@PAKPAU_CONTEXT@@PBU_s_FuncInfo@@PAXHK@Z 10036e04 f   LIBCMTD:frame_ce.obj
 0001:000363a0       ?CanThisExceptionObjectBeDestructed@@YAEPAUEHExceptionRecord@@E@Z 100373a0 f   LIBCMTD:frame_ce.obj
 0001:0003662c       ?BuildCatchObject@@YAXPAUEHExceptionRecord@@PAKPBU_s_HandlerType@@PBU_s_CatchableType@@@Z 1003762c f   LIBCMTD:frame_ce.obj
 0001:0003697c       ?AdjustPointer@@YAPAXPAXABUPMD@@@Z 1003797c f   LIBCMTD:frame_ce.obj
 0001:000372e8       ??__EgModem@@YAXXZ         100382e8 f   swiusb.obj
 0001:00037354       ??__FgModem@@YAXXZ         10038354 f   swiusb.obj

 Exports

  ordinal    name

        1    ?DriverEntry@@YAJPAU_CEDRIVER_OBJECT@@PAU_UNICODE_STRING@@@Z (long __cdecl DriverEntry(struct _CEDRIVER_OBJECT *,struct _UNICODE_STRING *))
               exported name: DriverEntry
        2    ?QMI_Close@@YAHPAUQMI_OPEN_INFO@@@Z (int __cdecl QMI_Close(struct QMI_OPEN_INFO *))
               exported name: QMI_Close
        3    ?QMI_Deinit@@YAHPAUQMI_PORT_MDD@@@Z (int __cdecl QMI_Deinit(struct QMI_PORT_MDD *))
               exported name: QMI_Deinit
        4    ?QMI_IOControl@@YAHPAUQMI_OPEN_INFO@@KPAEK1KPAK@Z (int __cdecl QMI_IOControl(struct QMI_OPEN_INFO *,unsigned long,unsigned char *,unsigned long,unsigned char *,unsigned long,unsigned long *))
               exported name: QMI_IOControl
        5    ?QMI_Init@@YAPAXPB_WPBX@Z (void * __cdecl QMI_Init(wchar_t const *,void const *))
               exported name: QMI_Init
        6    ?QMI_Open@@YAPAXPAXKK@Z (void * __cdecl QMI_Open(void *,unsigned long,unsigned long))
               exported name: QMI_Open
        7    ?QMI_Read@@YAKPAXPAEK@Z (unsigned long __cdecl QMI_Read(void *,unsigned char *,unsigned long))
               exported name: QMI_Read
        8    ?QMI_Seek@@YAKPAXJK@Z (unsigned long __cdecl QMI_Seek(void *,long,unsigned long))
               exported name: QMI_Seek
        9    ?QMI_Write@@YAKPAXPAEK@Z (unsigned long __cdecl QMI_Write(void *,unsigned char *,unsigned long))
               exported name: QMI_Write
       10    ?SWD_Close@@YAHPAUSWD_OPEN_INFO@@@Z (int __cdecl SWD_Close(struct SWD_OPEN_INFO *))
               exported name: SWD_Close
       11    ?SWD_Deinit@@YAHPAUSWD_MDD@@@Z (int __cdecl SWD_Deinit(struct SWD_MDD *))
               exported name: SWD_Deinit
       12    ?SWD_IOControl@@YAHPAUSWD_OPEN_INFO@@KPAEK1KPAK@Z (int __cdecl SWD_IOControl(struct SWD_OPEN_INFO *,unsigned long,unsigned char *,unsigned long,unsigned char *,unsigned long,unsigned long *))
               exported name: SWD_IOControl
       13    ?SWD_Init@@YAPAXPB_WPBX@Z (void * __cdecl SWD_Init(wchar_t const *,void const *))
               exported name: SWD_Init
       14    ?SWD_Open@@YAPAXPAXKK@Z (void * __cdecl SWD_Open(void *,unsigned long,unsigned long))
               exported name: SWD_Open
       15    ?SWD_Read@@YAKPAXPAEK@Z (unsigned long __cdecl SWD_Read(void *,unsigned char *,unsigned long))
               exported name: SWD_Read
       16    ?SWD_Seek@@YAKPAXJK@Z (unsigned long __cdecl SWD_Seek(void *,long,unsigned long))
               exported name: SWD_Seek
       17    ?SWD_Write@@YAKPAXPAEK@Z (unsigned long __cdecl SWD_Write(void *,unsigned char *,unsigned long))
               exported name: SWD_Write
       18    ?SWI_Close@@YAHPAUVSP_OPEN_INFO@@@Z (int __cdecl SWI_Close(struct VSP_OPEN_INFO *))
               exported name: SWI_Close
       19    ?SWI_Deinit@@YAHPAUVSP_PORT_MDD@@@Z (int __cdecl SWI_Deinit(struct VSP_PORT_MDD *))
               exported name: SWI_Deinit
       20    ?SWI_IOControl@@YAHPAUVSP_OPEN_INFO@@KPAEK1KPAK@Z (int __cdecl SWI_IOControl(struct VSP_OPEN_INFO *,unsigned long,unsigned char *,unsigned long,unsigned char *,unsigned long,unsigned long *))
               exported name: SWI_IOControl
       21    ?SWI_Init@@YAPAXPB_WPBX@Z (void * __cdecl SWI_Init(wchar_t const *,void const *))
               exported name: SWI_Init
       22    ?SWI_Open@@YAPAXPAXKK@Z (void * __cdecl SWI_Open(void *,unsigned long,unsigned long))
               exported name: SWI_Open
       23    ?SWI_PowerDown@@YAHPAX@Z (int __cdecl SWI_PowerDown(void *))
               exported name: SWI_PowerDown
       24    ?SWI_PowerUp@@YAHPAX@Z (int __cdecl SWI_PowerUp(void *))
               exported name: SWI_PowerUp
       25    ?SWI_Read@@YAKPAXPAEK@Z (unsigned long __cdecl SWI_Read(void *,unsigned char *,unsigned long))
               exported name: SWI_Read
       26    ?SWI_Seek@@YAKPAXJK@Z (unsigned long __cdecl SWI_Seek(void *,long,unsigned long))
               exported name: SWI_Seek
       27    ?SWI_Write@@YAKPAXPAEK@Z (unsigned long __cdecl SWI_Write(void *,unsigned char *,unsigned long))
               exported name: SWI_Write
       28    ?WMP_Close@@YAHK@Z (int __cdecl WMP_Close(unsigned long))
               exported name: WMP_Close
       29    ?WMP_Deinit@@YAHK@Z (int __cdecl WMP_Deinit(unsigned long))
               exported name: WMP_Deinit
       30    ?WMP_IOControl@@YAHKKPAEK0KPAK@Z (int __cdecl WMP_IOControl(unsigned long,unsigned long,unsigned char *,unsigned long,unsigned char *,unsigned long,unsigned long *))
               exported name: WMP_IOControl
       31    ?WMP_Init@@YAKPB_WPBX@Z (unsigned long __cdecl WMP_Init(wchar_t const *,void const *))
               exported name: WMP_Init
       32    ?WMP_Open@@YAKKKK@Z (unsigned long __cdecl WMP_Open(unsigned long,unsigned long,unsigned long))
               exported name: WMP_Open
       33    ?WMP_PowerDown@@YAXK@Z (void __cdecl WMP_PowerDown(unsigned long))
               exported name: WMP_PowerDown
       34    ?WMP_PowerUp@@YAXK@Z (void __cdecl WMP_PowerUp(unsigned long))
               exported name: WMP_PowerUp
       35    ?WMP_Read@@YAKKPAXK@Z (unsigned long __cdecl WMP_Read(unsigned long,void *,unsigned long))
               exported name: WMP_Read
       36    ?WMP_Seek@@YAKKJG@Z (unsigned long __cdecl WMP_Seek(unsigned long,long,unsigned short))
               exported name: WMP_Seek
       37    ?WMP_Write@@YAKKPBXK@Z (unsigned long __cdecl WMP_Write(unsigned long,void const *,unsigned long))
               exported name: WMP_Write
       38    USBDeviceAttach
       39    USBInstallDriver
